:100000002BC03AC039C038C037C0D1C035C034C0A9
:1000100033C032C031C030C02FC02EC02DC055C03B
:100020005EC068C071C07BC07FC083C08CC001024D
:100030000000040000000000010204081020200459
:100040001008020202020202020202020000000084
:10005000380000000000370011241FBECFE5D2E0B9
:10006000DEBFCDBF20E0A0E6B0E001C01D92A93602
:10007000B207E1F7E1D1EBC1C3CF85B5816085BDA2
:100080000895CF93DF93EC0160E080E067D160E0FA
:1000900080E09DD160E081E061D160E081E097D1B6
:1000A00060E082E05BD160E082E091D160E083E0DB
:1000B00055D160E083E08BD1C830D10508F050C045
:1000C000FE01E15FFF4F61E0099480E047D161E00C
:1000D00080E07DD161E081E041D160E009C080E055
:1000E0003DD160E080E073D161E081E037D161E033
:1000F00081E033C081E032D161E081E068D161E02C
:1001000082E02CD160E009C081E028D160E081E08C
:100110005ED161E082E022D161E082E01EC082E037
:100120001DD161E082E009C082E018D160E082E088
:100130000EC080E013D161E080E049D161E083E04E
:100140000DD160E009C080E009D160E080E03FD1DE
:1001500061E083E003D161E083E0DF91CF9137C1BB
:10016000DF91CF910895CF93DF93C0E0D0E0CE012F
:1001700088DF62E370E080E090E087D02196C830AD
:10018000D105A9F7C7E0D0E0CE017BDF62E370E0E4
:1001900080E090E07AD02197B8F78FEF9FEF71DF82
:1001A00068EE73E080E090E0DF91CF916EC01F9227
:1001B0000F920FB60F9211242F933F938F939F931B
:1001C000AF93BF938091610090916200A091630012
:1001D000B09164003091600020E3230F2D3720F4AC
:1001E0004096A11DB11D05C023EB230F4196A11D13
:1001F000B11D209360008093610090936200A093F2
:100200006300B09364008091650090916600A091B6
:100210006700B09168000196A11DB11D8093650033
:1002200090936600A0936700B0936800BF91AF9170
:100230009F918F913F912F910F900FBE0F901F9024
:1002400018953FB7F8948091650090916600A09151
:100250006700B091680022B708B601FE05C02F3FC5
:1002600019F00196A11DB11D3FBF6627782F892F78
:100270009A2F620F711D811D911D46E0660F771F39
:10028000881F991F4A95D1F708958F929F92AF9238
:10029000BF92CF92DF92EF92FF926B017C01D1DF90
:1002A0004B015C01C114D104E104F104E1F0CED0B2
:1002B000C8DF681979098A099B09683E734081057E
:1002C000910580F321E0C21AD108E108F10888EE17
:1002D000880E83E0981EA11CB11CC114D104E10456
:1002E000F10431F7DFCFFF90EF90DF90CF90BF9018
:1002F000AF909F908F90089578948AB582608ABD60
:100300008AB581608ABD83B7826083BF83B781600D
:1003100083BF89B7826089BF80B7826080BF32980F
:10032000319A309A379A0895823081F018F48130EA
:1003300051F00895833019F0843009F008958CB598
:100340008F7D8CBD08958AB58F7702C08AB58F7D69
:100350008ABD08958CB580648CBD0895CF93DF93DA
:1003600090E0FC01E85CFF4F2491FC01EE5BFF4F45
:100370008491882349F190E0880F991FFC01EE5A7F
:10038000FF4FA591B491845B9F4FFC01C591D4911F
:100390009FB7611108C0F8948C91209582238C93AB
:1003A000888182230AC0623051F4F8948C91322FF4
:1003B000309583238C938881822B888304C0F894A2
:1003C0008C91822B8C939FBFDF91CF9108950F93D7
:1003D0001F93CF93DF931F92CDB7DEB7282F30E066
:1003E000F901E25DFF4F8491F901E85CFF4F149140
:1003F000F901EE5BFF4F04910023C1F0882319F04F
:10040000698392DF6981E02FF0E0EE0FFF1FE45B6C
:10041000FF4FA591B4919FB7F8948C91611103C0DF
:100420001095812301C0812B8C939FBF0F90DF918A
:10043000CF911F910F9108955FDF8CDF1EDEC0E02A
:10044000D0E091DE2097E9F3DBDDFBCF0895F8944F
:02045000FFCFDC
:00000001FF
